:1010000000000000DD240600029A0800C90000006C
:041010008FAD0000A0
:10800000B240805A20013F401C000F9305242F836B
:108010009F4F9C920011FB233F4054010F93042477
:108020001F83CF431C11FC233040908830403080A8
:1080300000134E4F5D421D007DF00F007FF0F0FFFA
:108040004DDFC24D1D00F2D21D007EF00F005F42D9
:108050001C007FF0F0FF4FDEF2C21D007FF33041C5
:108060004E4F0E5E0E5E0E5E0E5E12C34F104F112F
:108070004F114F114FDE7FF330410B120A124A4F5E
:108080004B4E7FF220245F421D007FF0F1FF4E4AED
:108090007EF006004FDEC24F1D006AB20320F2D010
:1080A000F0FF1E004F4BB01232804B4F4F4A5FE340
:1080B0005FF311244F4BB0126080B0123280B012C7
:1080C00060804B4F083C4E437F400C00B0127A80DA
:1080D0004F93F93BD83FF2F00F001E004F4B3A414F
:1080E0003B4130410E4FE2E331008F107FF3B0127D
:1080F0007A807FF330410B120A123F40983AB01257
:108100006A8B3F403009B012E4803F408813B012C0
:108110006A8B3F403009B012E4803F40E803B01260
:108120006A8B3F403208B012E4803F402800B01212
:10813000E4801F43B012E4803F400600B012E480A8
:108140003F400C00B012E4803F404000B012E48099
:108150003B4000113A4017116E4B1B536F43B01256
:108160007A800B9AF927F82B3A413B4130410B12A8
:108170000B4F6E4B1B534E9304246F43B0127A8007
:10818000F83F3B4130410B120B4EB012E4800F4BD5
:10819000B0126E813B413041252B302A64000B1216
:1081A0000A120912081207120B4F0A4E074D094C0A
:1081B000084E0F12295309122983301298810E128A
:1081C000B012748B0A5F31520B930320F8402000E9
:1081D000000009930C240E4A1E530F4A3A53EF4AEB
:1081E00000003953FA23FA400A0000000A4E0F4AF1
:1081F0000F880F970834FA40200000001A530F4AE6
:108200000F880F97F83BCA43000037413841394186
:108210003A413B4130410E4FE2C219008F107FF3CB
:10822000C24F7700C24E77005F4271005FE35FF399
:10823000FB23E2D2190030410B120A1209120A4E36
:108240000B4F094D0F4E3FF0FF3F0FDDB01216826E
:108250000E4A0F4B8E108F104EEF0EEF8F110F1135
:108260000E100F110E100F110E100F110E100F1116
:108270000E100F110E1009DE0F49B012168239418F
:108280003A413B4130413F402020B01216823D40F0
:1082900000401E4230111F423211B012388230416C
:1082A000924220113011924222113211D2D3700029
:1082B000F240E2FF7100E2437400C2437500C24322
:1082C0007300F2401F007000F2D040000400D2C3DF
:1082D0007000F2D00A001B00B012868230410B12EF
:1082E0005B431E4230111F4232111E5228111F6281
:1082F0002A11824E3011824F32111C4224111D422C
:1083000026110C8E0D7F07349242201130119242BB
:10831000221132114B43B01286824F4B3B41304108
:108320000F125F4234127FF33F503411DF427E0060
:108330000000D25334123F410013D2D37800C2431D
:1083400035125F423512C24F3412C2437C00F240F4
:108350000F007D00C2437800D2C378003041D2D3F1
:108360007800F24020007900F24028007C00C243EF
:108370007D00C2437B00F24010007800F2D0300054
:108380000500D2C37800F2D0C0FF1B00F2D010006D
:108390000100B2400A002201B2407F00E4013041F6
:1083A0000D433D530F245E4235125F4234124E9FFF
:1083B000F8275F4235127FF35F4F3411D2533512E5
:1083C0007FF330413F4330410B120A1209120B4E2A
:1083D0000A4F09430E930A24B012A0833F93062448
:1083E000CA4F00001A5319533B53F6230F49394122
:1083F0003A413B4130412801244D44433032383822
:108400005C30303331343135395C4D4F44454D5C4F
:108410004D4443303134342C41544D303039365C86
:108420005A495020323838433429B240F683E201A9
:10843000B2403400E601B240F003E001B2B2E00124
:10844000FD273F43B0126A8BB0125E8330410F129A
:108450000E120D120C120B120A1209120812071238
:10846000E2E23100194240011952460119524C0111
:10847000195252011952361218424201185248013B
:1084800018524E011852540118523812F25010006E
:1084900046125742461277B0300021204E475EF315
:1084A0001A24E2E3310067B3922412C309100911C0
:1084B00009110911C249471289104F487FF0F0FF96
:1084C0004FD9C24F48120F488F107FF3C24F491245
:1084D000B240F003E001084309434E937020824903
:1084E0003612824838121942440119525001195269
:1084F0003A124F477FF070007F9020001724824986
:108500003A1219424A0119523C12184256011852A5
:108510003E120F473FF0F0003F906000702082490C
:1085200042128248441208430943693C824940127E
:108530001842181108930824385382481811022051
:1085400082494A120943DB3F1F424A1212C30F10ED
:108550000F110F110F110C490A4FB01254923C9099
:1085600010002B280E4C3E50F0FF084E1F422C11DD
:10857000099F212C0C4F0C8912C30C100C110C11EB
:108580000C9E012C084C0F483F5010003C420A4FF3
:10859000B01254920F4C0F93032408581F83FD23ED
:1085A0003892012C38423890DD0002283840DC0037
:1085B00082487601C73F0C43E33F0E43D63FB012DB
:1085C000DE824F938C23F2F0FCFF4612883F1F425D
:1085D0005012099F082C82495012924230114C12BD
:1085E000924232114E1282995612752F82495612BA
:1085F0009242301152129242321154126C3F82490F
:108600003C1282483E123741384139413A413B41A0
:108610003C413D413E413F410013B2435012824331
:108620005612B2404712E201B2400300E601C2DF37
:1086300046123041D2D331007F400300B0121A8677
:10864000D2B34612FD23D2C331003041423A205406
:10865000696D654F75742025642E00423A204F4B9A
:10866000202020202000423A204665686C65722157
:10867000000004123180100004413E4014003F40CD
:108680001C11B012C8833F90140019240F1230122D
:108690004C860412B012748B0E443F40C000B012DE
:1086A00086813D401C113E4000103F401400FD4EAD
:1086B00000001D531F83FB2331500600333C9242C0
:1086C0001C11C8011F421E113FE31F53824FCA01F4
:1086D0009242201130119242221132111E42241175
:1086E0001F4226111E8230111F7232110938B0123A
:1086F00086823E405B863F40C000B0128681123CBD
:108700003D4020113E4004103F400C00FD4E000053
:108710001D531F83FB233E4066863F40C000B012BE
:108720008681E53F3150100034413041B2401C1188
:10873000E201B2401400E601B240F003E001304132
:10874000B2404012E201B2400600E601B240F0033E
:10875000E00130410B120A120A4E0B4F021232C2D4
:10876000B0122C9232410E4F0F4E0F5F0F7F3FE33E
:108770000F4E3A413B4130410B120A1209120C4F85
:10878000094D0F430A4C0B430C4E0D4F0E4A0F4B35
:10879000B01254870F5939413A413B4130412B3F88
:1087A0003F2C3F3F6B487A203F3F3F2C3F56002BEA
:1087B0003F2C3F3F3F205620203F3F2C3FDF4300D0
:1087C0003E409E873F408000B01286813E40AF878A
:1087D0003F40C000B01286813041202050432D53CD
:1087E0007465756572756E08202000202020202099
:1087F0002020202020202020202020003E40DA873A
:108800003F408000B01286813E40EB873F40C00071
:10881000B01286813041202052657365742020207B
:10882000202020202020002020506E502D41626604
:10883000726108653F2020003E4016883F4080005E
:10884000B01286813E4027883F40C000B01286812A
:108850003041C29F58120B24C24F58125F930E240E
:108860006F9306386F9301243041B012388830413D
:108870004F9301243041B012C0873041B012FC87C1
:10888000304110121310121110121310129A2100FD
:1088900031400025F240E0FF5600F24087FF5700CC
:1088A000F24018005500B24049A52A01C2432100F8
:1088B000D2432200F24003002900F240FBFF2A00CD
:1088C000F2405C001900F2405F001A00C2431D0034
:1088D000F2400F001E00C2433100F240BFFF3200E1
:1088E000C2433500F24337003D401C113E400010AA
:1088F0003F401400FD4E00001D531F83FB233D40ED
:1089000080003E4082883F400C00FD4E00001D5319
:108910001F83FB23B2400004A601B2401602A2014D
:10892000B240F322A001B240B203C001B240B20390
:10893000C20192421C11C8011F421E113FE31F5386
:10894000824FCA01B240FF007201B24010026001C2
:10895000B240E0006601F2D010002E00B012F680A6
:10896000B0125E83F2B0200018000224B0123A83E5
:108970006F43B0125288B012A08232D2F2B010000F
:108980007800E424B012A0833F904200D9243F90A5
:108990004300C4343F9361243F9041005824C29364
:1089A0005812EC232C433D4006003E4059121F4212
:1089B0006612B0129E813E4059123F408000B012B4
:1089C00086810D433E409C041F424012B0127887BE
:1089D000824F68121C433D4006003E405912B012BF
:1089E0009E813E4059123F408900B01286810D435E
:1089F0003E40EC091F424212B01278873C4003000F
:108A00003D4006003E405912B0129E813E40591230
:108A10003F40C000B01286813D40AEFC3E404C0954
:108A20001F424412B0127887824F6A121C433D40A5
:108A300005003E405912B0129E813E4059123F40FF
:108A4000C900B01286813F43B0126A8B973F5F43E3
:108A5000B0125288B0123486A23FD29358123724F3
:108A60004F43B0125288B24002F8CA013F4000049E
:108A7000B0126A8B5F43B0121A86D2B34612FD233E
:108A80001A4252121B425412B240FE07CA013F4022
:108A90000004B0126A8B5F43B0121A86D2B346123A
:108AA000FD231F421E113FE31F53824FCA011E4286
:108AB00052121F4254120A8E0B7F3C405B060D433C
:108AC0000E4A0F4BB0125487824F6612683F3D40EA
:108AD00014003E401C113F400010B012FC910F9357
:108AE000BF27B24000A52C01B24002A52801B24325
:108AF0000010B24040A528013D4000103E401C112E
:108B00003F401400FD4E00001D531F83FB23B24065
:108B100000A52801B24010A52C01A23F3F904300C0
:108B200009243F9044003B235F43B0125288B012A7
:108B30004087353F5F43B0125288B0122C872F3FD9
:108B40005F43B0125288B0127286293FF2B0200003
:108B5000180025233E408E883F40CD00B01286810C
:108B6000B0122A841C3F30409A920F9302241F8334
:108B7000FE2330412F430F512C4F1E4F02002F5226
:108B80000D4F0F4CB0129A8B30411E426C12CE4FDB
:108B9000000092536C127FF330410B120B4F824F47
:108BA0006C123F408A8BB012188C0B5FCB430000D5
:108BB0003B4130410B120A120A4F0B4E0E9302201A
:108BC0001F430D3C6F4A8F111A5392126E120F936E
:108BD000053892531A113B53F523F23F3F433A4174
:108BE0003B4130410B120A120912494F4B4E5E9322
:108BF0000C384A4F8A110F4A92126E120F9307389F
:108C000092531A117B535B93F6374F49013C3F4314
:108C100039413A413B4130410B120A120912081204
:108C2000071206120512041231803C00054D8143E3
:108C300030008143320082431A11824F6E12064E79
:108C40000F46674647930A2477902500072416535A
:108C500067464793032477902500F9230D460D8F2F
:108C600002243040B091479302203040BE91165309
:108C7000C1432E00C1433500C1432F007B43C14394
:108C800028006746165377907500022030408A917D
:108C90004F477FD020007F907800022030408A919B
:108CA00077902000022030407691779023000220B8
:108CB00030406E9177902A00022030405291779098
:108CC0002D0002203040429177902B00022030404E
:108CD000389177902E0002203040D290779030006B
:108CE00002203040BC904F477F50CFFF7F9009005B
:108CF0001A2C0D430F4D0F5F0F5F0E4D0E5E0D4F83
:108D00000D5E0D5E0D5E4F478F110D5F3D50D0FF24
:108D1000674616534F477F50D0FF7F900A00EA2BDB
:108D2000C14D2F00B03F77906800C42577906C004C
:108D30000320D1D32E00A53F77906300B425779010
:108D40004400AE25779064007F25779069007C25EC
:108D500077904F00762577906F00702577907000A0
:108D60005E25779073001F25779055001925779021
:108D700075001225779058008F24779078008C2406
:108D8000479302203040BE9181412C00C147000032
:108D90005943C14328004B495A4135004A897A302A
:108DA0005E4128004E9370245B534B5A58412E006D
:108DB00078F0300013205D412F008D114F4B8F1143
:108DC0000D8F1D930B384E4D7F402000B012E48B69
:108DD0000F9302343040BE915E4128004E934F20E5
:108DE000F1B040002E0014241F412A003FF000FF84
:108DF0003FD03000814F2A00C1472B002E430F4146
:108E00003F502A00B012B48B0F9302343040BE9111
:108E10007890200024244E4A7F403000B012E48B2A
:108E20000F93CD394F498F110E4F1F412C00B012B7
:108E3000B48B0F93C439F1B010002E0001275D41AF
:108E40002F008D114F4B8F110D8F1D93F93A4E4D01
:108E50007F402000B012E48B0F93F236B03D5D41AD
:108E60002F008D114F4B8F110D8F1D93D43B4E4D05
:108E70007F403000B012E48B0F93CD37A03D1E43EE
:108E80000F413F502800BE3FF1B040002E008D271B
:108E90006B538B3F4A43843FF14010003400F1B2E2
:108EA0002E00092481933000032081933200032493
:108EB000F1D040002E00C1432800C14B35004B9338
:108EC0000338F1F0DFFF2E000F413F502800814FA3
:108ED0002C00819330000620819332000320C1933F
:108EE00035003E24D14134003800C143390081436C
:108EF0003A00C14336001E4130001F4132001E813E
:108F000038001F713A000228D14336001C4130005E
:108F10001D4132001A4138001B413A00B0127092D4
:108F2000444E7E900A00302C74503000B1532C0017
:108F30001F412C00CF4400001C4130001D41320075
:108F40001A4138001B413A00B0127092814C300037
:108F5000814D3200C1933600CC23F19234000624B7
:108F6000494159812C0079502800153FF1B22E005B
:108F7000F72774903000F427B1532C001F412C00C8
:108F8000FF4030000000EC3F7450570077905800CD
:108F9000CD2374F0DFFFCA3FF1400A0034008B3F5D
:108FA000D1D32E00F93F0F452553A14F2C008193BB
:108FB0002C001E244B9311384F4B8F110D4F0E4335
:108FC0001F412C00B012D8910F930524494F5981AD
:108FD0002C004B99DE36494BDC3E1F412C001F8391
:108FE0001F53CF930000FC23494F59812C00D13EE1
:108FF00081412C00F14028000000F1406E0001008A
:10900000F14075000200F1406C000300F1406C007B
:109010000400F14029000500C1430600CB3F0F4585
:109020002553A14F300081433200F140100034003D
:10903000F1D040002E00774078003D3FF1423400EF
:109040003A3FD1D32E00FA3FD1B32E0019240F4559
:109050002552B14F3000B14F3200819332000438B5
:10906000F1400A003400293FB1E33000B1E332009F
:109070009153300081633200F1402D002800F03F11
:109080000F452553A14F30009141300032009151DE
:1090900032003200917132003200B1E33200DD3F24
:1090A000D1D32E00D13F81412C000F452553E14FF4
:1090B00000006E3EE1D22E003040828CF1B01000F4
:1090C0002E0002243040828CF1D020002E0030404F
:1090D000828C6746165377902A0024240D434F470D
:1090E0007F50D0FF7F900A00162C0F4D0F5F0F5F4F
:1090F0000E4D0E5E0D4F0D5E0D5E0D5E4F478F11D6
:109100000D5F3D50D0FF674616534F477F50D0FF4D
:109110007F900A00EA2B0F4D3D9301343F434B4FA4
:109120003040868C0F4525532D4F0F4D3D93013414
:109130003F434B4F3040828CF1402B0028003040A1
:10914000828CF1D010002E00F1F0DFFF2E003040B5
:10915000828C0F452553E14F2F00C1932F00023819
:109160003040828CF1E32F00D1532F00EA3FF1D23F
:109170002E003040828CC193280002243040828C23
:10918000F140200028003040828CD1B32E0008240A
:109190000F452552B14F3000B14F32003040A08C06
:1091A0000F452553A14F3000814332003040A08C41
:1091B0000E4DB012B48B0F9302383040668C1F42B4
:1091C0001A1131503C003441354136413741384164
:1091D00039413A413B4130410B120B4F4C4E0D93FC
:1091E00007240E4B6F4E1E534F9C04243D53FA230D
:1091F0000F43023C0F4E3F533B4130410B120B4D8E
:109200000D930A240C4F0D4E6E4D1D536F4C1C5385
:109210004F9E04203B53F8230C43053C5C4CFFFF5E
:109220005F4DFFFF0C8F0F4C3B413041824C3001B2
:10923000824A3801824C34011E423A0192423C017A
:109240003A01824B3801824D3401824A38011F4273
:109250003A0130410EEE3B401100053C0D100E6E00
:109260000E9A01280E8A0C6C0D6D1B83F72330417A
:109270000FEF0EEE394021000A3C08100E6E0F6F02
:109280000F9B052802200E9A02280E8A0F7B0C6C79
:0C9290000D6D08681983F1233041FF3F89
:10929C0000000F11110F010E00001E11111E1010F5
:0C92AC0000000000000C04084006000058
:10FFE0002C802C802C8020832C802C802C804E8494
:10FFF0002C802C802C802C802C802C802C800080CD
:040000030000800079
:00000001FF
